:1000000000308A00E22A00000A108A100A118207D2
:1000100028340C34013406340A108A100A1182077D
:1000200025345834203458343D3425346C34643409
:10003000203459343D3425346C3464342034543401
:100040004C3431343D342534553454344C3432340A
:100050003D3425345534203454344C3433343D3419
:1000600025345534003434308400000803194728FF
:100070000130F800F701F70B3B28F80B3A284A301B
:10008000F700F70B412800000000800B38280034EF
:100090000608F039BB003A080F393B048600851486
:1000A0008316851000008312851083168510831235
:1000B0000034B808031D5E2805105F280514831658
:1000C00005108312B90E3908BA004820B90E390854
:1000D000BA0048200D30F700F70B6C2800341430BC
:1000E000B4003320F0308316860583120510831682
:1000F000051083128510831685108312AB012B081F
:10010000023C031C8B280230B40033200330BA00B9
:100110004820AB0A7F280D30F700F70B8D280230FE
:10012000BA0048200D30F700F70B9428AB012B08DC
:10013000023C031CA7282B080420AC00B8012C08A3
:10014000B90059200230B4003320AB0A97288A1135
:10015000242BAD0183168616061383120613213055
:10016000F700F70BB12883168612831286128316C6
:1001700006178312061BB728AC012C08073C031C8A
:10018000DA28831606178312061BC1282B18CA28E3
:100190008612CB2886168316861283122B08013905
:1001A000AD070310AB0C831606178312061FD32866
:1001B000AC0ABD28831606178312061BDA282D0801
:1001C000FF3A0139003A031DE7288612E82886160F
:1001D0008316861206178312061BF0288316EA2858
:1001E0008316861686168312861EF8288316F22832
:1001F000831606178312061BF82883160617831228
:10020000061FFD28831686168312861EFD280034DD
:1002100001303402B6003508023C031D112940307C
:10022000B60736088038B700B8013708B90059203A
:10023000003433080C3A03192729063A03192F29E9
:10024000073A03193529053A03193A293F29B80114
:100250000130B90059200230B40033204B2901305D
:10026000B4000230B50008214B290130B400B500BC
:1002700008214B29B8011030B90059204B29330807
:100280001F3C031C45290730B3050130B800330873
:10029000B90059204B290034AC1B5E290F30F70000
:1002A0002B0EF7050A307702031859293030F7076B
:1002B0005B292C08F7077708B30019210F30AB052D
:1002C0000A302B020318662930306829AC132C0839
:1002D000AB072B08B30019218A11372B0408B20091
:1002E000AC1F7B292D30B30019218403AB09AC0965
:1002F000AB0A0319AC0A2C0EF038AE00AE07E23E92
:10030000AF00323EB1002C080F39AF07AF07B1077D
:10031000E93EB000B007B0072B0E0F39B007B107A8
:10032000B00DB10DB109B10D2B080F39B107AE0DEC
:100330000730AD000A30B107B003031C9B29B0079A
:10034000AF03031C9F29AF07AE03031CA329AE070D
:10035000AD03031CA7292D30840007303205840724
:10036000313004020319D0290008F700031DBE290B
:10037000321ACE29B219C0292030C1290830B20062
:100380003030F707AC010408AB007708AD00770800
:10039000B30019212B0884002D08F700840AB02926
:1003A0000008F7003030F7077708B3001921003450
:1003B0003208F80131020318E0293108F700EC296E
:1003C000F7010830B300B10DF70D320877020318BA
:1003D000F700F80DB30BE32900343013B0122F08E7
:1003E000B1006430B200D8217708AF007808031D4F
:1003F000172AB01A172AB019252A301B052A3018D7
:10040000052A3019052AB01B252A301C112AB01BD9
:10041000252A301B112A3018252A3019112AB01B21
:10042000252A2030301E3030B3001921252AB0167D
:10043000B01F212A78088000F8002D30B300192160
:10044000B01330307807B3001921301B302A2F0841
:10045000B1000A30B200D8217708AF003017F62972
:10046000B01F352A2D30B300192130302F07B300CB
:10047000192100343510831606178312061B3B2AF8
:10048000831686168312861A3B2A83160617831252
:10049000061F452AB301B4013408073C031C7C2A1B
:1004A000831606178312061B502A0310B30C8316FB
:1004B000861600308312861A0130F700770CF70198
:1004C0000318F7177708B304003035180130B60069
:1004D0008316861600308312861A01303606F8001D
:1004E0007818742A3510752A351483160617831266
:1004F000061F752AB40A4C2A831606178312061B98
:100500007C2A003035180130B6008316861600307C
:100510008312861A01303606F8007818912A3510B1
:10052000922A3514831606178312061F922A831601
:1005300006178312061B972A831606178312061FB7
:100540009C2A3308F80000343A227808B0003A2296
:100550007808B1003A227808B20030080839083C1F
:10056000031DB82A2B0884003108003C8000BC2AF7
:100570002B0884003108800030081039103C031D1E
:10058000C72A2C0884003208003C8000CB2A2C08A3
:100590008400320880002D08840030080139800072
:1005A0002E0884000310300C013980002F088400CD
:1005B000300CF700F70C3F30F70577080139800061
:1005C0008A11A52B84011F30830583161F129F12E9
:1005D0001B0880399B0007309C001C0883120D13F8
:1005E000603083168F008312A101A201A301A40130
:1005F00083161F129F121B0880399B0083121F1045
:100600009412831606118614061200308312940089
:10061000831694000108C7390838810083129001BD
:100620000030F800920000308316920007309C00E2
:1006300005080330F700F70B1B2B1C0883120D1362
:1006400083169D0183126F280230AB00FA30B4008C
:100650003320AB0B262BF030AB00A9200130B400C7
:10066000B50008212508AB003730AC004C292030FC
:10067000B30019215830B30019213D30B3001921BE
:10068000103084002208AC002108AB006E2120301D
:10069000B30019215930B30019213D30B30019219D
:1006A000103084002408AC002308AB006E210E300B
:1006B000AB002B080C20AB0AF700B3001921133054
:1006C0002B02031D592B2808AF001830B000ED2174
:1006D0000330AC002030B3001921AC0B6A2B15306D
:1006E000AD002D080C20AD0AF700B3001921193018
:1006F0002D02031D712B2908AF001830B000ED2129
:100700001B30AE002E080C20AE0AF700B3001921F2
:1007100020302E02031D822B2A08AF001830B000B3
:10072000ED211430B4003320EB30AB00A9203A2285
:100730007808A5002630AB002730AC002830AD008B
:100740002930AE002A30AF00A42AFA012608A61BE1
:10075000FA03A1070318A20A7A08A207FA012708D8
:10076000A71BFA03A3070318A40A7A08A4072E2BD1
:02077000630024
:04400E00783FFF3FB9
:00000001FF
